S02000002E2E5C62696E5C6F70656E626C745F73746D3332663330332E73726563AF
S315080000000030002065110008B3110008B51100087A
S31508000010B7110008B9110008BB110008000000005C
S31508000020000000000000000000000000BD110008EC
S31508000030BF11000800000000C1110008C311000824
S31508000040C5110008C7110008C9110008CB1100081E
S31508000050CD110008CF110008D1110008D3110008EE
S31508000060D5110008D7110008D9110008DB110008BE
S31508000070DD110008DF110008E1110008E31100088E
S31508000080E5110008E7110008E9110008EB1100085E
S31508000090ED110008EF110008F1110008F31100082E
S315080000A0F5110008F7110008F9110008FB110008FE
S315080000B0FD110008FF1100080000000001120008E9
S315080000C003120008000000000000000005120008E6
S315080000D00000000007120008091200080B120008A9
S315080000E00D1200080F1200080000000000000000B2
S315080000F000000000000000000000000000000000F2
S3150800010000000000000000000000000000000000E1
S315080001100000000000000000111200081312000879
S3150800012000000000000000000000000000000000C1
S3150800013000000000000000000000000000000000B1
S315080001401512000817120008000000000000000041
S315080001500000000000000000000000000000000091
S315080001600000000000000000000000000000000081
S315080001700000000000000000000000000000000071
S31508000180000000001912000810B5054C237833B991
S31508000190044B13B10448AFF300800123237010BD4C
S315080001A09C00002000000000C41A0008084B10B587
S315080001B01BB108490848AFF300800848036803B92B
S315080001C010BD074B002BFBD0BDE81040184700BFF9
S315080001D000000000A0000020C41A00089C000020AF
S315080001E000000000154B002B08BF134B9D46A3F5D6
S315080001F0803A00218B460F461348144A121A01F01A
S3150800020007FC0F4B002B00D098470E4B002B00D055
S3150800021098470020002104000D000D48002802D050
S315080002200C48AFF3008001F0CDFB2000290000F058
S31508000230A1FC01F0B3FB00BF00000800003000205D
S3150800024000000000000000009C000020A40500201B
S31508000250000000000000000008B500F045F84FF463
S3150800026000714FF0904000F027F9034600B10123D2
S31508000270184608BD08B5642000F006F808BD00BF9A
S3150800028008B500F007F808BD014B1880704700BF95
S31508000290BC00002008B501F009F80F4B1B6898420E
S315080002A018D30E4B1B783BB901220C4B1A70082148
S315080002B00B4800F009F906E00022084B1A700821DD
S315080002C0074800F003F900F0F1FF064B1B881844B5
S315080002D0014B186008BD00BFB8000020BE00002012
S315080002E000040048BC00002008B50821014800F0B9
S315080002F0EDF808BD00040048054B1B6913F0800F94
S3150800030005D0034B034A5A6002F188325A60704797
S315080003100020024023016745024A136943F080031F
S315080003201361704700200240014BD860704700BF38
S31508000330002002400B4BDB6813F0010F0BD1094B71
S31508000340DB6813F0100F08D1064BDB6813F0040FB7
S3150800035005D003207047012070470220704704200B
S31508000360704700BF0020024010B50446FFF7E2FFC1
S3150800037002E0FFF7DFFF013C012801D1002CF8D18C
S3150800038004B9052010BD00BF38B505464FF4302026
S31508000390FFF7EAFF042811D1094C236943F0020349
S315080003A023616561236943F0400323614FF43020DC
S315080003B0FFF7DAFF236923F00203236138BD00BF84
S315080003C00020024030B583B005460C460023019351
S315080003D04FF43020FFF7C8FF042820D1114A1369CB
S315080003E043F001031361A3B22B804FF43020FFF7CB
S315080003F0BBFF04280ED102350195019B240C1C80F5
S315080004004FF43020FFF7B0FF064A136923F00103C3
S31508000410136104E0034A136923F00103136103B06F
S3150800042030BD00BF0020024070B400233FE0012227
S315080004309A400C68A24339D10A79013AD2B2012A04
S315080004401CD885685A000324944025EA040484606D
S3150800045085684C7904FA02F22A4382608488A5B238
S315080004609AB20124944025EA040484808588ADB2B2
S315080004708C7904FA02F22A4392B2828004685A00FE
S31508000480032505FA02F624EA0604046006680C79D0
S31508000490944034430460C4689EB27600B54024EAAA
S315080004A00505CC7904FA02F22A43C26001330F2B00
S315080004B0BDD970BC704700BF038A194201D001201C
S315080004C070470020704700BF8161704701857047FB
S315080004D030B401F007039B009A40C908083150F868
S315080004E021400F2505FA03F324EA030340F82130D7
S315080004F050F821301A4340F8212030BC704700BF1D
S31508000500F0B5A04B5B6803F00C03042B06D0082B50
S3150800051008D003BB9C4B036000241FE09A4B036082
S3150800052000241BE0974B5C685A68C4F38344A31CF9
S3150800053012F4803F03D1954C04FB03F409E0914A79
S31508000540D26A02F00F0201328F4CB4FBF2F404FBBC
S3150800055003F4046002E08C4B03600024894D6B6849
S31508000560C3F30313DFF828E21EF80370FFB202682C
S3150800057022FA07F343606968C1F302211EF80110E5
S31508000580C9B223FA01F181606E68C6F3C2261EF865
S315080005900660F6B2F340C360ED6A2D0905F00F0C4C
S315080005A0DFF8F0E13EF81CE01FFA8EFE15F0100F9A
S315080005B006D0BEF1000F03D0B4FBFEF5056100E0DE
S315080005C00261704DED6A6D0A05F00F0CDFF8C4E1A3
S315080005D03EF81CE01FFA8EFE15F0100F06D0BEF18D
S315080005E0000F03D0B4FBFEF5456100E04261654D9E
S315080005F02D6B15F0100F02D1634D856100E0826105
S31508000600604D2D6B15F0200F02D15F4DC56100E0DE
S31508000610C2615C4D2D6B15F0400F02D15A4D056233
S3150800062000E00262574D2D6B15F4807F06D0944288
S3150800063004D1B74202D16500456200E04362514DDC
S315080006402D6B15F4805F06D0944204D1B74202D1CF
S315080006506500856200E083624A4D2D6B15F4007FC4
S3150800066006D0944204D1B74202D16500C56200E0C3
S31508000670C362444D2D6B15F4806F06D0944204D1A5
S31508000680B74202D16500C56400E0C3643D4D2D6BD9
S3150800069015F4006F06D0944204D1B74202D1650022
S315080006A0056500E00365374D2D6B15F4005F06D030
S315080006B0944204D1B74202D16500456500E003655E
S315080006C0304D2D6B15F4004F06D0944204D1B74235
S315080006D002D16400846500E083652A4B1B6B13F026
S315080006E0030F01D1816319E0264B1B6B03F003034B
S315080006F0012B01D1826311E0224B1B6B03F003032C
S31508000700022B03D14FF40043836307E01D4B1B6B99
S3150800071003F00303032B01D11B4B8363194B1B6B9C
S3150800072013F4403F01D1C1631CE0164B1B6B03F465
S315080007304033B3F5803F01D1C26313E0114B1B6B05
S3150800074003F44033B3F5003F03D14FF40043C363CA
S3150800075008E00C4B1B6B03F44033B3F5403F01D163
S31508000760094BC363074B1B6B13F4402F01D101647C
S3150800077026E0044B1B6B03F44023B3F5802F0BD103
S3150800078002641DE00010024000127A0000093D00D4
S3150800079020000020000000202E4B1B6B03F4402392
S315080007A0B3F5002F03D14FF40043036408E0294B47
S315080007B01B6B03F44023B3F5402F01D1264B03648A
S315080007C0244B1B6B13F4401F01D141641CE0214BE1
S315080007D01B6B03F44013B3F5801F01D1426413E089
S315080007E01C4B1B6B03F44013B3F5001F03D14FF4E6
S315080007F00043436408E0174B1B6B03F44013B3F53F
S31508000800401F01D1144B4364124B1B6B13F4400F6A
S3150800081001D18164F0BD0F4B1B6B03F44003B3F5A4
S31508000820800F01D18264F0BD0A4B1B6B03F44003B1
S31508000830B3F5000F03D14FF400438364F0BD054BB5
S315080008401B6B03F44003B3F5400F01D1024B8364DD
S31508000850F0BD00BF0010024000127A0021B1054B1E
S315080008605A69104358617047024A536923EA0000DF
S31508000870506170470010024021B1054BDA691043F8
S31508000880D8617047024AD36923EA0000D0617047ED
S315080008900010024030B599B004460D46036823F0AF
S315080008A001030360436823F440528B681343436093
S315080008B0036823F4B05222F00C024968EB68194326
S315080008C02B690B4313430360836823F440726B69F7
S315080008D01343836001A8FFF713FE1C4B9C4201D10A
S315080008E00F9A0FE01A4B9C4201D1109A0AE0194B55
S315080008F09C4201D1119A05E0174B9C4201D1129AEC
S3150800090000E0139A236813F4004F06D052002968B2
S31508000910B2FBF1F301FB132204E02968B2FBF1F301
S3150800092001FB13222968B2EB510F00D30133226869
S3150800093012F4004F06D0C3F3420223F00F031B0440
S315080009401B0C13439BB2A38119B030BD003801407C
S315080009500044004000480040004C004021B10368B4
S3150800096043F0010303607047036823F00103036043
S31508000970704700BFC1F3080101857047808CC0F33A
S3150800098008007047C3690B4201D001207047002058
S31508000990704700BF1222164B1A60A3F580535A6897
S315080009A05A605A685A605A6842F480625A605A68AD
S315080009B022F47C125A605A6842F460125A601A6825
S315080009C042F080721A600B4B1B6813F0007FFAD056
S315080009D0084B5A6822F003025A605A6842F002022B
S315080009E05A60044B5B6803F00C03082BF9D1704777
S315080009F0002002400010024008B5144B1A6842F065
S31508000A0001021A605968124A0A405A601A6822F0A6
S31508000A10847222F480321A601A6822F480221A60DC
S31508000A205A6822F4FE025A60DA6A22F00F02DA6283
S31508000A30196B084A0A401A6300229A60FFF7AAFF50
S31508000A404FF00062044B9A6008BD00BF00100240D8
S31508000A500CC07FF8CCFC00FF00ED00E02DE9F0416A
S31508000A6082B001214FF48020FFF7F8FE4FF0080806
S31508000A70CDF8008001248DF8044000258DF8065035
S31508000A8003268DF805608DF80750394F69463846B4
S31508000A90FFF7CAFC41463846FFF718FD21464FF4D2
S31508000AA00030FFF7DBFE8DF804508DF807404FF451
S31508000AB00073009369464FF09040FFF7B5FC214656
S31508000AC04FF40030FFF7D8FE21464FF40030FFF709
S31508000AD0C5FE072202214FF09040FFF7F9FC0722D6
S31508000AE00F214FF09040FFF7F3FC8DF806508DF874
S31508000AF0074002278DF80470042300938DF80560DB
S31508000B0069464FF09040FFF78FFC8DF804704FF45C
S31508000B100043009369464FF09040FFF785FC214655
S31508000B204FF40030FFF79AFE09220B214FF0904050
S31508000B30FFF7CEFC09220C214FF09040FFF7C8FCC6
S31508000B404FF4C05300938DF804708DF805608DF846
S31508000B5006508DF8074069464FF09040FFF764FC51
S31508000B6021464FF00070FFF787FE02B0BDE8F0811E
S31508000B700004004808B5FFF771FF00F08BFC00F091
S31508000B8097FCFCE7F0B5002422E0134D15F814E0B5
S31508000B9005EB44056F780EEB070606FB00064FF4D7
S31508000BA0FA4595FBF6F506FB05F5B5F5FA4F0DD1B1
S31508000BB095FBF6F6B6B20E80013EB6B2B6F5806F74
S31508000BC004D282F800E01F700120F0BD0134E4B2BF
S31508000BD0112CDAD90020F0BD641A000800B583B0DC
S31508000BE001AB0DF105020DF106014FF4FA70FFF79E
S31508000BF0C9FF012803D0E221384800F01BFC384B16
S31508000C0000225A611A6842F400421A6001E000F0B4
S31508000C10C9FC334B1B6813F4004FF8D1304B1A68E4
S31508000C2022F002021A601A6842F001021A6001E014
S31508000C3000F0B8FC2A4B5B6813F0010FF8D09DF85A
S31508000C4005305A1E9DF80430013B1B0543EA024352
S31508000C50BDF80620013A1343214AD361136823F0ED
S31508000C600103136001E000F09DFC1D4B5B6813F067
S31508000C70010FF8D11A4BD3F8002242F00102C3F84B
S31508000C800022D3F81C2222F00102C3F81C22D3F852
S31508000C900C2242F00102C3F80C220022C3F84022BB
S31508000CA0C3F84422D3F8042222F00102C3F804222E
S31508000CB0D3F8142222F00102C3F81422D3F81C2216
S31508000CC042F00102C3F81C22D3F8002222F00102E6
S31508000CD0C3F8002203B05DF804FB00BF3C1A000805
S31508000CE00064004038B504460D46214B9B6813F056
S31508000CF0806F04D140F221111E4800F09BFB1C4B6B
S31508000D00D3F8802102F00102C3F88021D3F88021AC
S31508000D1042F07C4242F40012C3F88021C3F88451A1
S31508000D20E178A278120442EA0162617842EA012275
S31508000D3021780A43C3F88821E179A279120442EAA4
S31508000D400162617942EA012221790A43C3F88C21BA
S31508000D50D3F8802142F00102C3F8802101E000F0B7
S31508000D6021FC034B9B6813F0806FF8D038BD00BF99
S31508000D70006400403C1A00081B4BDB6813F0030FA5
S31508000D802FD0194BD3F8B02140F26763B3EB525F0B
S31508000D9020D1154BD3F8B8210270D3F8B821120A1E
S31508000DA04270D3F8B821120C8270D3F8B821120E0B
S31508000DB0C270D3F8BC210271D3F8BC21120A427161
S31508000DC0D3F8BC21120C8271D3F8BC311B0EC37147
S31508000DD0012000E00020044AD36843F02003D360D2
S31508000DE070470020704700BF0064004008B500F057
S31508000DF0B5F908BD10B500F021FAA0B1FFF72CFA35
S31508000E0088B100F08BFB00F02BFA00F01BFA20F0FB
S31508000E10604020F07F00044B186000F013FA446825
S31508000E2000F09EF9A04710BD08ED00E070B508E097
S31508000E30461C4D1C0B78037000F0B4FB2246304666
S31508000E402946531E9CB2002AF2D170BD08B5C1F3DB
S31508000E50080353B90368994209D040F8041B4FF4B4
S31508000E600072FFF7E3FF012008BD002008BD01203E
S31508000E7008BD00BF2DE9F0410746FFF73DFA3420CB
S31508000E80FFF752FAFFF756FA012815D100241BE09E
S31508000E903E68A30006EB03083B445D6800F082FB4E
S31508000EA029464046FFF78EFA04280AD156F8243018
S31508000EB09D4208D1013400E000247F2CE8D90124A2
S31508000EC002E0002400E00024FFF726FA2046BDE8E9
S31508000ED0F08100BF38B50D460B4B984207D0044643
S31508000EE00A4B994205D0FFF7C5FF18B908E0084C28
S31508000EF000E0054C29462046FFF7A8FF10B938BD83
S31508000F00002038BD204638BDC0000020002000085B
S31508000F10C40200202DE9F04106460C4617461D4638
S31508000F2021F4FF7828F001080368B3F1FF3F04D1E4
S31508000F304146FFF78BFF034630B33368984505D023
S31508000F4041463046FFF7C6FF0646D0B13368E41A75
S31508000F503444043400F026FB331DE31AB3F5007F4E
S31508000F6007D308F500713046FFF7B4FF064650B1BF
S31508000F70041D17F8013B04F8013B013DEAD10123A2
S31508000F8002E0002300E000231846BDE8F08100BF18
S31508000F904FF0FF33024A1360024A1360704700BFDE
S31508000FA0C4020020C00000200E4B984216D910B586
S31508000FB04318013B0C4CA34212D80B46014620F4B9
S31508000FC0FF7020F00100094CA04203D10848FFF742
S31508000FD0A1FF10BD0748FFF79DFF10BD0020704711
S31508000FE0002010BDFF1F0008FFFF000800200008B2
S31508000FF0C0000020C402002070B520F4FF6525F06B
S3150800100007051A4B9D422DD94318013B184A9342AE
S315080010102AD8401B0144C1F3CF26C1F30A0109B1FE
S315080010200136B6B2FFF768F93420FFF77DF9FFF706
S3150800103081F901280CD1002410E000F0B3FA05EB81
S31508001040C420FFF7A1F9042807D10134A4B200E0AF
S315080010500024A642F1D8012400E00024FFF75CF939
S31508001060204670BD002070BD002070BDFF1F00081F
S31508001070FFFF0008114B1B68B3F1FF3F18D000B5FE
S3150800108083B00E4B59689A681144DA6811441A6994
S3150800109011445A6911449A691144DA698B185B42FA
S315080010A002AA42F8043D04210548FFF77DFF01E046
S315080010B00120704703B05DF804FB00BFC0000020A4
S315080010C0882100080D4B1A6804331B6813440C4A20
S315080010D0126813440B4A126813440B4A11680B44EE
S315080010E0043212681A44094B1B681344084A1268EA
S315080010F0D34201D101207047002070470020000824
S31508001100082000080C2000081020000818200008F5
S315080011108821000808B50D4B1B68B3F1FF3F04D0C2
S315080011200A48FFF7A7FE034668B1094B1B68B3F1E7
S31508001130FF3F05D00648FFF79DFE034610B902E0BB
S31508001140012300E00123184608BD00BFC0000020A7
S31508001150C4020020004870470020000872B6704795
S3150800116062B6704707498D460749084A084B9A42AE
S31508001170BEBF51F8040B42F8040BF8E70548804750
S315080011800548004700300020D01A0008000000205B
S315080011909C000020F9090008E50100081F49204ABB
S315080011A0002301E041F8043B9142FBD3FFF7E2FC40
S315080011B0FEE7FEE7FEE7FEE7FEE7FEE7FEE7FEE7F9
S315080011C0FEE7FEE7FEE7FEE7FEE7FEE7FEE7FEE7E9
S315080011D0FEE7FEE7FEE7FEE7FEE7FEE7FEE7FEE7D9
S315080011E0FEE7FEE7FEE7FEE7FEE7FEE7FEE7FEE7C9
S315080011F0FEE7FEE7FEE7FEE7FEE7FEE7FEE7FEE7B9
S31508001200FEE7FEE7FEE7FEE7FEE7FEE7FEE7FEE7A8
S31508001210FEE7FEE7FEE7FEE7FEE700009C0000208B
S31508001220A405002008B5FFF7B3FE08BD08B5FFF70B
S31508001230BBFE08BD08B5FFF7DFFE08BD08B5FFF71A
S3150800124041FF08BD08B5FFF785FF08BD08B5FFF7DC
S3150800125011FF034610B1FFF75DFF0346184608BDA8
S315080012600022014B1A60704710E000E008B5FFF74E
S31508001270F7FF054B4FF6FF125A6000229A600521C8
S315080012801960024B1A6008BD10E000E0C80400208F
S31508001290044B1B6813F4803F03D0034A13680133D9
S315080012A01360704710E000E0C804002008B5FFF797
S315080012B0EFFF014B186808BDC804002010B50446A6
S315080012C080210948FFF75EFB58B121460648FFF71B
S315080012D051FB80210448FFF755FB0028F9D001206F
S315080012E010BD002010BD00BF0044004010B50446E4
S315080012F020210648FFF746FB012805D10348FFF7DA
S315080013003DFB2070012010BD002010BD00440040A8
S3150800131010B586B04FF461430093002301930293FE
S31508001320039305930C230493054C69462046FFF75F
S31508001330B1FA01212046FFF711FB06B010BD00BF28
S315080013400044004070B506460D46402903D975216C
S315080013500F4800F06FF82846FFF7B0FF012803D0C2
S3150800136079210B4800F066F800240CE000F01AF921
S31508001370305DFFF7A3FF012803D08221044800F05F
S3150800138059F80134A4B2ABB29C42EFD370BD00BF8A
S31508001390881A000838B5224B1C789CB92148FFF7F3
S315080013A0A5FF01283AD11F4B1B78002B31D0FFF738
S315080013B07DFF1D4B186000221C4B1A700122184B2A
S315080013C01A702BE00546194B1B780133154818444B
S315080013D0FFF78CFF0446012810D1144B1A78013206
S315080013E0D2B21A700F4B1B789A4214D1104928466C
S315080013F0FFF71CFD00220A4B1A700FE0FFF756FF95
S31508001400094B1B686433984207D90024044B1C70A7
S3150800141004E01C4602E0002400E00024204638BD13
S3150800142011050020D0040020CC040020120500205D
S31508001430D104002008B500F0B5F8FCE708B500F0BF
S31508001440A9F8012810D0094B1B78012B0CD1FFF7FE
S315080014502DFF074B1B6803F5FA73984204D3002245
S31508001460024B1A70FFF7C6FC08BD00BF1305002023
S315080014701405002008B50122044B1A70FFF716FF61
S31508001480034B1860FFF7DAFF08BD00BF13050020FD
S315080014901405002008B5FFF7A9FC00F07FF8FFF750
S315080014A0E5FEFFF7BFFE00F00DF8FFF7E3FF08BD06
S315080014B008B500F077F8FFF7EBFE00F013F8FFF732
S315080014C0BDFF08BD10B500F0DBF9FFF787FB044C3C
S315080014D001232370FFF71CFF0023237010BD00BFF4
S315080014E03000002008B50B48FFF746FC012805D157
S315080014F00122094B1A70074800F0E0F90548FFF782
S3150800150049FF012805D10022034B1A70014800F053
S31508001510D5F908BD1805002030000020704700BF27
S3150800152038B504460D46084B1B78012B02D1C9B2C3
S31508001530FFF7D8FB044B1B781BB9E9B22046FFF727
S3150800154001FF00F0B3F938BD30000020074B1B78C7
S31508001550022B05D0032B05D0012B05D04020704760
S315080015600020704700207047082070473000002090
S31508001570074B1B78022B05D0032B05D0012B05D072
S3150800158040207047002070470020704708207047A9
S315080015903000002008B500F081F908BD08B5FEF74F
S315080015A069FE08BD08B5FEF76BFE08BD10B400233A
S315080015B004E010F8011B0B44DBB221464C1E00293F
S315080015C0F7D11360012010BC704700BF0022014B01
S315080015D05A70704758050020034BFE22DA701871BE
S315080015E00222A3F8442070475805002010B5054C80
S315080015F000232370FFF7EAFFFF23E3700123A4F813
S31508001600443010BD58050020064BFF22DA70002230
S315080016101A71597859719A71DA711A720622A3F8F1
S31508001620442070475805002008B50020FFF7D4FF6E
S3150800163008BD00BF084BFF22DA70084A9A640022E8
S315080016401A715A719A710721D9711A725A729A7255
S315080016500822A3F84420704758050020B41A000849
S31508001660044BFF22DA7042689A640122A3F84420E8
S31508001670704700BF5805002010B5084CFF23E370DB
S31508001680E21D4168A06CFFF791FF2071002363718A
S31508001690A3710823A4F8443010BD00BF58050020E4
S315080016A008B53120FFF798FF08BD00BF38B5084CCC
S315080016B0FF23E370002525716571FFF747FFA071C9
S315080016C0E571257265720723A4F8443038BD00BF5A
S315080016D05805002038B5FFF779FF0E4C012525700F
S315080016E0FF23E3701023237100236371FFF72EFF96
S315080016F0A071FFF73DFFE071FFF73AFFC0F307203F
S3150800170020726572A5720823A4F84430FFF78AFD93
S3150800171038BD00BF5805002038B505464478FFF7A0
S3150800172015FF0138844203DD2220FFF755FF38BD37
S31508001730084C6A78A16C201DFFF778FBFF23E3703D
S315080017406B78A26C1344A3646B780133A4F8443015
S3150800175038BD00BF5805002038B504464578FFF760
S31508001760F5FE0138854203DD2220FFF735FF38BD37
S315080017706168084DA9646278281DFFF757FBFF23A7
S31508001780EB706378AA6C1344AB6463780133A5F8ED
S31508001790443038BD5805002038B505460D4B9C6CBD
S315080017A0FFF7D4FE6A1C411E2046FFF73FFD18B915
S315080017B03120FFF711FF38BD064CFF23E370FFF712
S315080017C0C5FE0138A36C1844A0640123A4F844306C
S315080017D038BD00BF5805002038B504464578FFF7E0
S315080017E0B5FE0238854203DD2220FFF7F5FE38BD37
S315080017F00F4BFF22DA700122A3F84420617831B931
S31508001800FFF724FD90B93120FFF7E6FE38BDA21C8C
S31508001810074B986CFFF70AFD18B93120FFF7DCFE75
S3150800182038BD6378024A916C0B44936438BD00BF97
S315080018305805002008B54168074B986CFFF7FAFC75
S3150800184018B93120FFF7C8FE08BD034BFF22DA702E
S315080018500122A3F8442008BD5805002008B5FFF763
S31508001860C9FA034BFF22DA700122A3F8442008BD07
S315080018705805002008B589B2FFF752FE08BD00BF1B
S31508001880054B00221A709A6483F84320A3F8442073
S315080018909A705A70704700BF58050020024B187896
S315080018A000B10120704700BF580500200022024BF6
S315080018B083F84320704700BF5805002008B5037811
S315080018C0FF2B02D1FFF706FF50E0334A1278012AB0
S315080018D060D1C93B352B46D8DFE803F0334545428E
S315080018E045453F363C3945454545454545454545C4
S315080018F0454545454545454545454545454545458A
S31508001900454545454545241E1B2145454527452A48
S315080019102D30FFF701FF29E0FFF71EFF26E0FFF74E
S315080019209FFE23E0FFF7A8FE20E0FFF783FE1DE0F9
S31508001930FFF77AFE1AE0FFF767FE17E0FFF756FE95
S3150800194014E0FFF729FF11E0FFF746FF0EE0FFF767
S31508001950ADFE0BE0FFF76EFF08E0FFF77FFF05E03F
S31508001960FFF79EFE02E02020FFF736FE0A4B93F8AB
S315080019704330012B02D11020FFF72EFE064BB3F998
S315080019804410002906DD1846012380F84330033049
S31508001990FFF770FF08BD00BF5805002008B5074BC4
S315080019A0044613B10021AFF30080054B1868836A1B
S315080019B003B19847204600F033F800BF0000000046
S315080019C0C01A000870B50E4B0E4CE41AA410002578
S315080019D01E46A54204D056F8253098470135F8E743
S315080019E000F020F8084C094BE41AA41000251E46FE
S315080019F0A54204D056F8253098470135F8E770BD5A
S31508001A0094000020940000209800002094000020F4
S31508001A1002440346934202D003F8011BFAE77047D3
S31508001A20FEE70000F8B500BFF8BC08BC9E46704744
S31508001A30F8B500BFF8BC08BC9E4670472E2E5C2E33
S31508001A402E5C2E2E5C2E2E5C536F757263655C4180
S31508001A50524D434D345F53544D333246335C6361C4
S31508001A606E2E630005020602060307030803090330
S31508001A7009040A040B040C040C050D050E050F05D4
S31508001A800F061006100710082E2E5C2E2E5C2E2E22
S31508001A905C2E2E5C536F757263655C41524D434DE7
S31508001AA0345F53544D333246335C756172742E631A
S31508001AB0000000004F70656E424C54004300000061
S30D08001AC03400002000000000BC
S30D08001AC81CE7FF7F0100000086
S31508001AD0010002000400060008000A000C001000BD
S31508001AE02000400080000001000000000000000007
S31508001AF000000000010203040102030406070809A6
S31508001B0004000000000000000000000000000000C3
S31508001B1000000000000000000000000000000000B7
S31508001B2000000000BC1A00080000000000000000C9
S31508001B300000000000000000000000000000000097
S31508001B400000000000000000000000000000000087
S31508001B500000000000000000000000000000000077
S31108001B6000000000AD0100088901000823
S70508000000F2
